:1000000012C034C01895189518951895189518951C
:100010001895189518951895189518951895189578
:100020001895189518958FED8DBFC0ECE0EC4E2E0D
:10003000DD275D2EEEE7F0E0A0E6B0E088278D93A7
:100040003197E9F766248CE387BB8BEF81BB80E0B7
:1000500088BB80E082BB929A959A78948BB7806433
:100060008BBF85B7806385BF8895FBCF0F921F92AA
:100070002F923F924F925F927F92AF92BF920F93D7
:100080001F932F933F934F935F936F937F938F9320
:100090009F93AF93BF93CF93DF93EF93FF938FB76C
:1000A0008F9384E690E07AD1829919C0959888E27E
:1000B00090E074D1C49AC59A8AE090E06FD1C59857
:1000C0008AE090E06BD1C498C59A8AE090E066D14E
:1000D000C598B79901C021D0B79B01C08CD08F9132
:1000E0008FBFFF91EF91DF91CF91BF91AF919F9122
:1000F0008F917F916F915F914F913F912F911F91C0
:100100000F91BF90AF907F905F904F903F902F9056
:100110001F900F9018950895C4CF80E080936100E0
:10012000009161000F3110F009F057C080E080931A
:10013000600080E08093620000916200073010F060
:1001400009F01BC0A0E60C9142E057D14C930091FE
:100150006000A6E38C9186FB882780F9482F040F66
:10016000A0E60C93C59A8AE090E018D1C598A2E663
:100170008C918F5F8C9308F4DFCFB0990AC000E2B6
:10018000A6E38C9181FB882780F9482F36D1A3E61E
:100190004C93B09B0EC000E2A6E38C9181FB8827B4
:1001A00080F9482F2AD1A3E64C93A3E68C91805C7A
:1001B0008C930091630040916100040FA3E60C93BF
:1001C000A3E6EC91FF27A0E691E07BE7FED0A1E655
:1001D0008C918F5F8C9308F4A3CF80E088BB959AB5
:1001E0008FEF8093640081E080936600ACD08299A9
:1001F00001C0FDCF089580E080936100009161000F
:100200000F3110F009F078C080E08093600080E04A
:100210008093620000916200073010F009F018C06E
:10022000A0E60C9142E0E9D04C9300916000A6E377
:100230008C9186FB882780F9482F040FA0E60C9349
:10024000C59AC598A2E68C918F5F8C9308F4E2CF93
:10025000A1E6EC91FF27A5E691E0C8D040916500AA
:1002600000916000041709F401C001C03FC0009173
:10027000610040E2040FA3E60C93A3E6EC91FF2794
:10028000A5E691E0B3D040916500009160000417AD
:1002900009F401C001C02AC00091610040E4040FCC
:1002A000A3E60C93A3E6EC91FF27A5E691E09ED090
:1002B0004091650000916000041709F401C001C07D
:1002C00015C00091610040E6040FA3E60C93A3E67D
:1002D000EC91FF27A5E691E089D04091650000915F
:1002E0006000041709F401C020C000C0A1E68C9191
:1002F0008F5F8C9308F482CF80E088BB959A8FEF54
:100300008093640081E0809366001DD0829901C0D3
:10031000FDCFE1E0F0E033D0949AE2E0F0E02FD0BE
:100320009498E1E0F0E02BD0089580E088BB959AA6
:100330008AE58093640089E08093660004D0829906
:1003400001C0FDCF089580E0809361004091660078
:1003500000916100041710F009F010C0939AA4E610
:100360008C9199271BD09398A4E68C91992716D04D
:10037000A1E68C918F5F8C9308F4E8CF089588EE06
:1003800093E00CD03197D9F708953197F1F708959C
:10039000689462F80895E89462F80895EF93FF93E3
:1003A000EE27E82BE92B31F0EAEFF0E03197F1F797
:1003B0000197D1F7FF91EF910895E199FECFEEBB40
:1003C0003196089591E001C092E07B3751F47FB7F8
:1003D000F894F3DF8D918DBBE29AE19A9A95C9F773
:1003E0007FBF7727089591E001C092E0E6DFE09AB1
:1003F0008DB38D939A95D1F70895FF935527F8E023
:10040000469508F4500F57954795FA95D1F7FF9107
:0204100008954D
:00000001FF
